:020000020000FC
:1000000009C018954AC12CC11895189518951895CE
:10001000189518950FE90DBF00E00EBBE09A0DB3DF
:100020000F3F09F001BFE0E6F0E0EF01112700E427
:1000300019930A95E9F736E0112400270283038318
:1000400000E10287002708BB0FE007BB02E009BF01
:1000500003E00FBD01E003BF00E20BBF00E105BB01
:1000600000E003B900E204BB00E007B907EC06B901
:1000700078940681002311F0363011F5363049F0BE
:1000800036E00FB50F750FBD002708BB0AE0202E24
:10009000F0CF06810023D1F3F89412812381789464
:1000A000163202E0200790F31B3802E0200770F7B9
:1000B0002220F9F6F78218E522E01483258375C023
:1000C000349903C03730E1F32DC014B125B1408518
:1000D0005185140F251F10872187349A369A02857F
:1000E0000A9511F00287EECF04E010852185269550
:1000F00017950A95E1F700270087018700E102873D
:10010000373059F0173D00E0200760F40FB50F7548
:100110000FBD002708BB37E0D3CF1C3201E020071A
:1001200078F2AECF0F2D1781011B043100F1F78259
:10013000F89442815381789414812581411B520B9C
:10014000B1F018F41150204002C01F5F2F4F1483EC
:100150002583113F00E0200758F4353041F0C29864
:10016000C0980FB50F7D0FBDC19AC39A35E081CFFE
:10017000163202E02007A8F4343051F0C2980FB5CF
:100180000F770FBDC0980FB500620FBDC39A34E062
:1001900046E252E0411B520B142F252F30D049BDAF
:1001A00068CF1B3802E0200758F4313041F0C39883
:1001B000C2980FB50F750FBDC09AC19A31E059CFE3
:1001C000103C03E0200790F4323051F0C3980FB593
:1001D0000F7D0FBDC1980FB500680FBDC29A32E008
:1001E0001A5802E0200B0BD046BF43CFC398C198EA
:1001F0000FB50F770FBDC09AC29A35E03ACF4CEDDC
:1002000050E09924882400E15695479510F4810E1A
:10021000921E97948794579547950A95B9F716E3D8
:1002200021E0EE24AA24CC24DD24BB1801E2441FE3
:10023000551F881C991C0A9589F0AA1CBB1CCC1C54
:10024000DD1CA11AB20ACE08DE0830F4A10EB21EDF
:10025000CE1CDE1C8894EBCF0894E9CF4D5D089549
:10026000DFB7DF93F394332021F0D181DF1509F458
:100270003324DF2DD37059F41394D12DD83C38F0AA
:1002800011243324D681DD2311F0DA95D683222080
:1002900009F02A94DF91DFBF1895BFB7BF93BBB7B2
:1002A000BF7DBBBF8F2D72B7B8B7B1FF02C072B7A9
:1002B00083957894B49B0DC03320A1F5B681B233F9
:1002C00019F4B12DB23370F170838183B1E03B2E0C
:1002D00029C0B49927C03324C08191817C1B890B2C
:1002E00086957795869577957835B2E08B07D0F02F
:1002F000703BB4E08B07F8F0705BB4E08B0B7830A8
:10030000B7E08B0778F4703BB4E08B0788F4C281C8
:1003100093817C0F891F869577957283838311243F
:10032000B2E3B683BBB7B062BBBFBF91BFBF189586
:0C03300070EB84E0ECCF70EB84E0E9CFD0
:00000001FF
